:1000000008308A0000280000FF00030E8301A100D1
:100010000A08A0008A010408A2007708A300780853
:10002000A4007908A5007A08A6007B08A70083131E
:1000300083128C308400801D1F288C1932282208DE
:1000400084002308F7002408F8002508F900260892
:10005000FA002708FB0020088A00210E8300FF0E0B
:100060007F0E09008A110A12BE280A108A100A118E
:10007000820728340C34013406340A108A100A111D
:1000800082070C34573465346C3463346F346D3408
:100090006534213420342E3420342E3420342E3450
:1000A0000A3400340A108A100A11820730343D34B1
:1000B000253475342034203431343D3425347534BE
:1000C000203432343D3425347534203400340A1061
:1000D0008A100A118207543465346D3470346534E3
:1000E000723461347434753472346534203430348D
:1000F0002034253432342E343134673400340A103D
:100100008A100A118207543465346D3470346534B2
:10011000723461347434753472346534203431345B
:100120002034253432342E343134673400340A100C
:100130008A100A118207543465346D347034653482
:10014000723461347434753472346534203432342A
:100150002034253432342E343134673400341308DB
:10016000831664088312930014168C1183161418D6
:10017000B728F8018312141AF80A00348316941A67
:10018000C6288312EE011318EE17831683126E0829
:10019000EE0AAB002B087F3C031CD128AB08031DE3
:1001A000D128B4013408083C031CE9280130340785
:1001B0002B02031DE7288316141CDC288312130866
:1001C000AA002C303407840083132A088000B40A64
:1001D000D2282B08803C031D2A292C08B500B40125
:1001E0003408203C031C2A2934083502031D0B293E
:1001F0000310340CF7000310F70D7708463E840017
:100200008313840A00088316E10084030008E000D9
:10021000E4008312AF20013034073502031D272983
:100220000310340CF7000310F70D7708463E8400E6
:100230008313840A00088316E10084030008E000A9
:100240006108E200E3016108E4008312AF2002309C
:10025000B407F0288C118A110A121F28D0308400AC
:1002600083130008031941290630F800F701F70B42
:100270003729F80B36297B30F700F70B3D29800B27
:1002800034290034831657184929831206124B2942
:1002900083168312061683160612D7185329831263
:1002A00086125529831683128616831686125719CD
:1002B0005D29831206135F2983168312061783169E
:1002C0000613D719672983128613692983168312A7
:1002D0008617831686130000061183120615033055
:1002E000F700F70B712983160611831206110034EB
:1002F00083168611831286116330F700F70B7E296F
:1003000081298316D40803198A2986118312861538
:100310008D2983168611831286110000831606111B
:10032000831206118316550ED6000F30D6055608D7
:10033000D70083124221831655080F39D600D70003
:100340008312422100340130A900831686118312E2
:100350008611831606118312061123308316D000EE
:1003600083122E218316C1014108023C031CC429BB
:100370000330D7008312422105308316D000831248
:100380002E218316C10AB4290230D70083124221DC
:100390008316C1014108033C031CE0294108831274
:1003A00035208316C200D4014208D500831278217B
:1003B00005308316D00083122E218316C10ACA2964
:1003C00083128A150A12402883165108013A8312B3
:1003D0000319F429033A0319F729013A0319FB29F0
:1003E000073A0319FF29042A8316D201072A40304D
:1003F0008316D200072A14308316D200072A5430FD
:100400008316D200072A83128316D201072A0130ED
:100410005002D20752088038D300D4015308D500C7
:1004200083127821003483164F080C3A8312031983
:10043000202A063A03192E2A023A0319392A402A99
:100440008316D4010130D500831278210130A90030
:1004500002308316D00083122E21482AA90A0130C7
:100460008316D000831229088316D1008312E42159
:10047000482A8316D4011030D50083127821482AE7
:1004800001308316D4004F08D50083127821482A02
:1004900000348E30F70083164408F8004308F90052
:1004A000FA01F808031D5E2A7908F800F9010830FE
:1004B000F702F808031D5E2AF701662A0310F81BED
:1004C000652AF90DF80DF7035E2AF81383128A15D1
:1004D0000A1292298030831C702A8316D406831254
:1004E0008316D901DA015008D8005408D8064F08FD
:1004F00003195E2BD700F70053080319672BD702A7
:100500000319032B031CC12A5408DD00DD1755080D
:10051000DC005608DB00DA010310DD0CDC0CDB0C20
:10052000DA0CD70B8B2AD81F982A59147B2B591019
:1005300057105916D23084008313902B5912D81BB0
:10054000AB2A571CB62ADD0CDC0CDB0CDA0CF70AE4
:100550000319762BB62ADD1BB92A0310DA0DDB0D41
:10056000DC0DDD0DF7030319762BAB2A5917232B6E
:1005700059135008D800D81FBF2ADD176F2BDD1381
:100580006F2B5308D700F7004F08D7025008DD0043
:10059000DD175108DC005208DB00DA010310DD0C26
:1005A000DC0CDB0CDA0CD70BCD2AD81FDA2AD914D5
:1005B0007B2BD9105710D916D63084008313902B7B
:1005C000D912D81BED2A571CF82ADD0CDC0CDB0CE9
:1005D000DA0CF70A0319762BF82ADD1BFB2A031025
:1005E000DA0DDB0DDC0DDD0DF7030319762BED2A9B
:1005F000D917232BD9135408D800D81F012BDD1786
:100600006F2BDD136F2B5408DD00DD175508DC0060
:100610005608DB00D81F102BDD1359157B2B591101
:10062000DA015710D23084008313902BD81B392B5A
:100630005008D800571C232BDD0CDC0CDB0CDA0C2B
:10064000F70A0319762BDA1F342BDB0A031D342B30
:10065000DC0A031D342BDD0A031D342BDD0CDC0CFE
:10066000DB0CF70A0319762B591BB82AD91BFA2A77
:10067000582B8030DD06DD1F412B7B2B5408D80022
:100680004E2B5008D800DD08031D4E2BDC08031D3F
:100690004E2BDB08031D4E2BF7016F2BDD1B582B58
:1006A0000310DA0DDB0DDC0DDD0DF70B4E2B762B79
:1006B000D81F5C2BDD176F2BDD136F2B5308F70052
:1006C0005408DD005508DC005608DB006F2B4F088E
:1006D000F7005008DD005108DC005208DB005D081F
:1006E000F8005C08F9005B08FA00AE2BF701F8018E
:1006F000F901FA01AE2BDA01DB09DC09DD09DA09BF
:10070000DA0A031D892BDB0A031D892BDC0A031976
:10071000DD0A5918972AD918D92A59190F2B3E2BB7
:100720000008DB07031C9A2BDC0A031D9A2BDD0A49
:100730000319571484030008DC07031CA22BDD0AED
:100740000319571484030008801F803ADD0703183B
:100750005714591A9E2AD91AE02A162B83120034EC
:10076000831647080319762CD3004B080319762CFF
:10077000D302031CC02B7F30D3070318762CC62B63
:100780008130D302031C762C0319762C5308F70012
:10079000F801F901FA01D2014808D100D11749083E
:1007A000D0004A08CF001930D3004E08CF020318FA
:1007B000E92B0130D0020318E92BD1020318E92BF1
:1007C000D2020318E92BD20AD10AD00A4E08CF0769
:1007D0001B2C4D08D0020318042C0130D102031841
:1007E000042CD2020318042CD20AD10A4D08D007D7
:1007F0004E08CF07031C1B2CD00A031D1B2CD10A4B
:10080000031D1B2CD20A1B2C4C088038D102031864
:100810001A2C0130D20203181A2CD20A4C08803844
:10082000D1074D08D007031CF82BD10A031DF82B64
:10083000D20AF82B7A14D30B1E2C292C0310CF0DBF
:10084000D00DD10DD20D0310FA0DF90DF80DD40D08
:10085000D52B541C312C0310F80CF90CFA0CD40CC9
:10086000342CF7030319762CD41B5D2C0310CF0D09
:10087000D00DD10DD20D4E08CF020318492C0130F6
:10088000D0020318492CD1020318492CD202031CB0
:100890006C2C4D08D0020318542C0130D1020318DF
:1008A000542CD202031C6C2C4C088038D102031843
:1008B0005D2C0130D202031C6C2CFA0A031D6C2C37
:1008C000F90A031D6C2CF80A031D6C2CF70A031996
:1008D000762CF80CF90CFA0C4808D3004C08D30617
:1008E000D31F742CF8177A2CF8137A2CF701F8011F
:1008F000F901FA0183128A150A12202AF701F80178
:100900008316410803104218F707F70CF80CC218B9
:10091000F707F70CF80C4219F707F70CF80CC21997
:10092000F707F70CF80C421AF707F70CF80CC21A85
:10093000F707F70CF80C421BF707F70CF80CC21B73
:10094000F707F70CF80C83128A150A12512A83163E
:10095000CB010408CA004B10831B4B14440EF03823
:10096000C600C607E23EC700323EC90044080F3940
:10097000C707C707C907E93EC800C807C807430E2D
:100980000F39C807C907C80DC90DC909C90D4308E2
:100990000F39C907C60D0730C5000A30C907C8039B
:1009A000031CCE2CC807C703031CD22CC707C603E1
:1009B000031CD62CC607C503031CDA2CC5308400E3
:1009C000831307304A054A138407C9300402031908
:1009D0004A170008F700031DF52C4A1BF52C4A1A8C
:1009E000092DCA19F52C2030F82CCA154A123030BE
:1009F000F707C4010408C3004410831B441477089C
:100A0000CF008312132283164308840083134418F3
:100A10008317840A4A1FE52C831200348316450885
:100A2000F80144020318172D4408F700232DF7019D
:100A30000830C600C40DF70D450877020318F7000B
:100A4000F80DC60B1A2D831200347808831642085D
:100A5000C4006430C50083120E2577088316C200D7
:100A600078083030031D3B2DC31C442DC319442D81
:100A7000431A20303E2DC31143124314F80778085F
:100A8000CF008312132283164208C4000A30C50027
:100A900083120E2577088316C20078083030031DB4
:100AA000572DC3195D2D431C5D2D431A2030F807C7
:100AB0007808CF008312132283163030C207420811
:100AC000CF00831213220034F701F801F901FA0173
:100AD0008316D701D801D901DA0156085504540408
:100AE00053040319A32D2030DB000310CF0DD00DCC
:100AF000D10DD20DD70DD80DD90DDA0D56085A02E9
:100B0000031D8C2D55085902031D8C2D54085802C5
:100B1000031D8C2D53085702031C9D2D5308D7022B
:100B20005408031C540FD8025508031C550FD90252
:100B30005608031C560FDA020314F70DF80DF90DD1
:100B4000FA0DDB0B752DD73084008313831200342C
:100B500004088316C7004608C90003193B2E450840
:100B6000D2004408D1004308D0004208CF00D6018B
:100B7000D5012030D4008230D3004F0803192D2E28
:100B8000D700530803192D2ED7070318CE2D7F3019
:100B9000D702031C2D2E03192D2ED22D8130D707FD
:100BA00003182D2E5708F700F801F901FA01500833
:100BB000DB00DB175108DA005208D9001830D700E3
:100BC000D801591CFB2D5608FA07031CED2DF90A14
:100BD000031DED2DF80A0319D8175508F907031C52
:100BE000F42DF80A0319D8175408D100D117510869
:100BF000F8070318D817D80DF80CF90CFA0CDB0C11
:100C0000DA0CD90C0310D70BE02D0130F7070318CD
:100C10002D2EF81B122EDB0DFA0DF90DF80DF70332
:100C200003192D2EDB1F232EFA0A031D232EF90A8A
:100C3000031D232EF80A031D232EF80CF90CFA0CC1
:100C4000F70A03192D2E5008D8005408D806D81FCB
:100C50002B2EF817312EF813312EF701F801F90178
:100C6000FA017A08C5007908C4007808C30077083B
:100C7000C200C90BAF2D7E30F700F801C31BF81777
:100C8000F901FA0183104508D2004408D100430855
:100C9000D0004208CF007A08D6007908D50078083D
:100CA000D4007708D30083126A227A088316C5001D
:100CB0007908C4007808C3007708C2004508D2004C
:100CC0004408D1004308D0004208CF004F08B63C8A
:100CD000CF00FA015008D300D0170310D00CD10C6C
:100CE000D20CFA0CF90CF80CF70CCF0B6D2ED31FAD
:100CF000842EF709F809F909FA09F70A0319F80A1D
:100D00000319F90A0319FA0A7A08C5007908C40018
:100D10007808C3007708C200C51F9B2EC703C716FB
:100D2000C209C309C409C509C20A0319C30A0319C0
:100D3000C40A0319C50A3B30CE009A30CD00CA3030
:100D4000CC00CB010A30C90046080319C70A450880
:100D5000D2004408D1004308D0004208CF004E081A
:100D6000D6004D08D5004C08D4004B08D3008312A0
:100D7000642500088316C200840A0008C300840AA0
:100D80000008C400840A0008C500FD308407F70885
:100D9000031DDD2E460A49020319DD2E47080319FB
:100DA000DF2E0F3949020319D72E0318172FC71B3F
:100DB000172F471BDF2E2030112F2030C705C71EED
:100DC000EF2EC7124608031DC7037708C7002D3052
:100DD000CF008312132283164708F700C701460885
:100DE0004902031DFF2E7708C7002E30CF00831263
:100DF000132283164708F7002030C7050030303033
:100E0000C71E112FC7124608031DC7037708C70066
:100E10002D30CF008312132283164708F700C70135
:100E20003030F7077708CF008312132283164E085D
:100E3000D2004D08D1004C08D0004B08CF00D6019D
:100E4000D501D4010A30D300831264257A088316B1
:100E5000CE007908CD007808CC007708CB00C90B0C
:060E6000A72E83120034EE
:10100000840183131F308305813083169900A63035
:101010009800903083129800A8152808831687003E
:1010200083122816280883168700A03093003630D4
:101030008312940083161F149F141F159F110730ED
:101040009C00FF308312A800AC01AD01AE01AF01DE
:10105000B001B101B201B3015B30E6005C30E700E2
:101060005D30E8005E30E9005F30EA006030EB00A0
:101070006130EC006230ED000330EE008A11A329EC
:101080008A1583168C15C03083128B048316C00119
:101090004008103C031C58280310400D463E8400B5
:1010A0008313840A8001840340088000C00A482812
:1010B000C830D0008A1183122E218A150C30831675
:1010C000CF008A11831213228A1502308316C100C1
:1010D000FA30D0008A1183122E218A158316C10B93
:1010E0006828C10141088A1183123D208A15003801
:1010F000031984288316C10ACF008A118312132290
:101100008A1583167228831208308316C100FA30BC
:10111000D0008A1183122E218A158316C10B8728CD
:101120001F109F101F119F111F1383121F179F174E
:1011300083169F1383121F148316C0014008073CB7
:10114000031C342A400DF700F70DF70DF830F705B2
:1011500083121F08C73977049F0064308316D000BC
:101160008A1183122E218A1503108316400D363EF4
:101170008400831383121F151F19BC281E08FA0050
:1011800083161E088000840A7A0880000310400D30
:10119000463EC100C2010318C20A0310400D363E8C
:1011A00084008313840A0008C40084030008C30079
:1011B000440CFA00430CF900FA0CF90CFA0CF90C87
:1011C000FA0CF90CFA0CF90CFA0CF90C0330FA05CC
:1011D0007908C5007A08C6004108840083134218C4
:1011E0008317840A460880008403450880000310A2
:1011F000400D463E84008313840A0008C200840325
:101200000008C1004208013C03181329FF3A031DDE
:101210000D2941087F3C03181329663040078400DC
:101220008313643080000310400D463E8400831316
:10123000840A0008C20084030008C1004208023C7E
:10124000031C2D29031D282941081C3C031C2D29A2
:10125000663040078400831380010310400D463E32
:1012600084008313840A0008C20084030008C100BC
:101270004208013C03187D29FF3A031D4329410818
:101280001C3C03187D290310400D463E8400831347
:10129000840A0008C40084030008C3004408023C18
:1012A000031C7D29031D582943087F3C031C7D290D
:1012B00066304007C100C2010318C20A0310400D86
:1012C000463E84008313840A0008C4008403000897
:1012D000C3001C304302F7004408FA000230031C2C
:1012E0000330FA027708C5007A08C6004108840076
:1012F00083134218831745088000400DF700F70D4F
:10130000FC30F7057708A03EC100C2010318C20AED
:1013100066304007840083130008C401C3008A11AB
:101320008312492A8A1583164108840083134218C0
:10133000831777088000840A78088000840A790877
:101340008000840A7A088000400DF700F70DFC3019
:10135000F7057708A03EC100C2010318C20A400D7C
:10136000F700F70DFC30F7057708A03E84008313E3
:101370000008C300840A0008C400840A0008C500ED
:10138000840A0008C600C8010408C7004810831B6F
:10139000481483144608D2004508D1004408D00000
:1013A0004308CF00D601D5012030D4008330D300CC
:1013B0008A1183126A228A158316470884008313D0
:1013C000481883174108840083134218831777084D
:1013D0008000840A78088000840A79088000840AE2
:1013E0007A088000400DF700F70DFC30F70577080C
:1013F000A03EC100C2010318C20A400DF700F70D5C
:10140000FC30F7057708A03E840083130008C30072
:10141000840A0008C400840A0008C500840A000881
:10142000C600CA004508C9004408C8004308C700F0
:10143000CE01CD01CC018030CB008A118312B02BBC
:101440008A1583164108840083134218831777088E
:101450008000840A78088000840A79088000840A61
:101460007A088000C00A9E280C30CF008A118312AF
:1014700013228A1505308316D0008A1183122E217B
:101480008A15AD08031D872B8316C0014008023C56
:10149000031C7D2A0530C1004008C2008A11831256
:1014A0007E2C8A157808013E8316C100D0000130D9
:1014B000D1008A118312E4218A1503108316400D8E
:1014C000463E84008313840A0008C2008403000897
:1014D000C100103084004208C4004108C3008A11D2
:1014E0008312A7248A1520308316CF008A11831215
:1014F00013228A158316C00A462A0130D000023012
:10150000D1008A118312E4218A1530308316CF006E
:101510008A11831213228A153D308316CF008A1157
:10152000831213228A1566088316C2001B30C3007B
:101530008A11831225258A1504308316C1004108BB
:101540008A11831252208A158316C10AF700CF0030
:101550008A11831213228A15083083164102031D53
:101560009F2A831267088316C2001B30C3008A11AA
:10157000831225258A1520308316CF008A11831205
:1015800013228A1532308316CF008A118312132258
:101590008A153D308316CF008A11831213228A15D3
:1015A00068088316C2001B30C3008A1183122525E8
:1015B0008A1520308316CF008A11831213228A15D0
:1015C00001308316D0000330D1008A118312E42148
:1015D0008A151030840047088316C4008312460819
:1015E0008316C3008A118312A7248A15203083161C
:1015F000CF008A11831213228A1510308400490803
:101600008316C400831248088316C3008A1183120C
:10161000A7248A1520308316CF008A118312132243
:101620008A15103084004B088316C40083124A08C0
:101630008316C3008A118312A7248A1501308316EA
:10164000D0000430D1008A118312E4218A152C08BD
:101650008316C2001B30C3008A11831225258A1508
:1016600020308316CF008A11831213228A152D0889
:101670008316C2001B30C3008A11831225258A15E8
:1016800020308316CF008A11831213228A152E0868
:101690008316C2001B30C3008A11831225258A15C8
:1016A00020308316CF008A11831213228A152F0847
:1016B0008316C2001B30C3008A11831225258A15A8
:1016C00020308316CF008A11831213228A15300826
:1016D0008316C2001B30C3008A11831225258A1588
:1016E00020308316CF008A11831213228A15310805
:1016F0008316C2001B30C3008A11831225258A1568
:1017000064308316D0008A1183122E218A152D0B86
:10171000172C01308316D0000230D1008A118312B9
:10172000E4218A158316C10141088A1183126720BA
:101730008A158316C10AF700CF008A11831213227B
:101740008A150E3083164102031D942B013084004C
:101750002308C5002208C4002108C3002008C200D5
:101760000130C6008A118312A8258A15013083161C
:10177000D0000330D1008A118312E4218A15831628
:10178000C10141088A1183127F208A158316C10A7C
:10179000F700CF008A11831213228A150E308316A8
:1017A0004102031DC12B013084002708C500260813
:1017B000C4002508C3002408C2000130C6008A11F5
:1017C0008312A8258A1501308316D0000430D10079
:1017D0008A118312E4218A158316C10141088A11F6
:1017E000831297208A158316C10AF700CF008A1149
:1017F000831213228A150E3083164102031DEE2B2D
:10180000013084002B08C5002A08C4002908C30041
:101810002808C2000130C6008A118312A8258A1543
:1018200064308316D0008A1183122E218A152E0B64
:101830001E2C8316081083120814222C83160810FD
:10184000831208102F0B292C8316881083128814FA
:101850002D2C8316881083128810300B342C83169D
:10186000081183120815382C8316081183120811E9
:10187000310B3F2C8316881183128815432C831655
:10188000881183128811320B4A2C83160812831296
:1018900008164E2C8316081283120812330B552C8F
:1018A0008316881283128816592C83168812831285
:1018B0008812831608168312081A622CD701013089
:1018C000D600642CD701D601831688168312881A95
:1018D0006D2CD9010130D8006F2CD901D8018316A5
:1018E00008178312081B782CDB010130DA007A2CF0
:1018F000DB01DA01831688178312881B832CDD0134
:0E1900000130DC00852CDD01DC019C28630039
:02400E00723FFF
:00000001FF
